:1000000016EF00F0EA6A060EE96EEF500EE0080EF9
:10001000016E006A002EFED7012EFBD7190E006E6E
:10002000002EFED700D0EF2EF2D7000CF86AD09E3B
:10003000EA6AE96AC150C00BC16E070EB46EC150C6
:10004000C00B0F09C16EC050C00BC06EC09EC280F5
:10005000C28EC282C2B2FED7C29EC69A949A9488B9
:100060009496010EC66E000EC76ED190800ED56EAE
:10007000CD6A000ECA6E000ECB6E766E000E776EE5
:100080009484BD6A796AB66A070EB46E9750976E0B
:10009000140E006E002EFED70000B450A19CB56A6D
:1000A000929A899A040E056EFA0E066EABDF052E43
:1000B000FBD7929A898A040E056EFA0E066EA2DFAD
:0800C000052EFBD7EDD703006C
:020000040001F9
:08FFF800A004C407F807000093
:00000001FF
